:020000020000FC
:1000000012C05BC360C31895189549C3189518951D
:100010001895189518951895189518951895189578
:100020001895189518951FED1DBFF89410E012B99A
:1000300011E819B910E01BB918E01AB916E013B9A4
:1000400014E01ABB14E01BBB1DEF17BB10E018BB7C
:1000500013E311BB1FE712BB10E01EBD10E718B978
:1000600010E015BF10E019BF10E01BBF5FD25ED2D9
:100070005DD2C39A18E218BB49D2C39847D238E27E
:1000800063D238E061D231E05FD248D236E05CD250
:10009000F89488279927CC27DD273CE055D2E8E75C
:1000A000F7E0ABD1FF24909A949A959A11271DBD41
:1000B0001CBDCF3F61F0843018F0DA3060F007C02B
:1000C000833018F0DF3138F002C0D43620F010E76A
:1000D00015BFC09A88954427552717E327D21A954C
:1000E000459B02C0439501C053951030B9F74517A1
:1000F00098F0E8EEF7E081D1D39546D216ED1CB921
:1001000043D21CD2823040F4E8EFF7E011E067D12F
:10011000E8EFF7E012E063D137D210EC182B1CB9EE
:1001200033D210E41BBF10E819BF9598EFD1789433
:10013000913029F011E0180F90981EBD04C011E015
:10014000180F94981EBDFFCF803081F08A9505C0AE
:100150009927843008F015C08395E8E8F7E04DD181
:1001600051D1CC2711D214ED1CB90ED29BCF4CEB40
:100170005FE760E0A416B506C60668F4803059F063
:10018000E3CFE8EBF7E039D115E5C10FFDD110ED74
:100190001CB9FAD187CF913051F12DE101D224362B
:1001A00009F01EC028E0FCD1422F29E0F9D1522FDE
:1001B000FDD1741A850A920A2BE0F2D1422F2EE06B
:1001C000EFD1522FF3D1A41AB50AC20A22E1E8D125
:1001D000422F27E1E5D1522FE9D1D41AE50AF20ADC
:1001E000DF92EF92FF927F928F929F9203C0A4EAD8
:1001F000B3E202C0A4E6B1E248D1843051F08330CA
:1002000039F0823021F0813009F072D171D16DD195
:100210006CD171D1903041F063D16AD18827992790
:10022000F8D06AD0F8D13ECF49E95AE3662777275C
:10023000D416E506F606070750F491E041ED57E0C5
:10024000D416E506F606070708F0839512C040E8C5
:1002500056E968E9D416E506F606070730F010E11E
:10026000712E17E2812E99242BD1D3D045D0CC27E3
:10027000D2D1FF90EF90DF90AFE7BFE006D14D2DD8
:100280005E2D6F2D702FDA2CEB2CFC2CA3E0B8E048
:10029000FCD09F908F907F90D41AE50AF60A070B46
:1002A0003AF4E8EAF7E070D113ED1CB96DD10DC056
:1002B00007D1FF2411ED27E0D116E20648F0E0EB6C
:1002C000F7E062D112ED1CB95FD112E088D0EACE1E
:1002D000A0D068D059D110E8312A3CB855D110E9E6
:1002E000212A2CB851D110EA112A1CB84DD110EB9B
:1002F000012A0CB849D1D6CE30E826D11127611693
:10030000D9F55116B1F5411629F5311619F430E237
:1003100021D109C0843021F430E31CD13CE21AD150
:1003200030E3330D17D130E3320D14D1843049F46A
:1003300030E3310D0FD130E3300D0CD130E20AD172
:100340002EC03CE207D130E3310D04D130E3300D53
:1003500001D121C030E3340DFDD030E3330DFAD0AC
:1003600030E3320DF7D03CE2F5D030E3310DF2D07E
:1003700012C030E2EFD003C030E3360DEBD030E3F3
:10038000350DE8D030E3340DE5D030E3330DE2D065
:1003900030E3320DDFD030E2DDD035E7DBD036E4BC
:1003A000D9D0089530ECD0D01127311621F030E3A8
:1003B000330DD0D002C030E2CDD030E3320DCAD000
:1003C0003CE2C8D030E3310DC5D030E3300DC2D0AF
:1003D00030E2C0D03FE4BED03CEBBCD0089578E022
:1003E000113019F430E8B0D002C030ECADD0359106
:1003F000B1D07A957030D9F7089511E0F0DF12E0AE
:10040000EEDF089537E8A0D030E3380F3395A2D05F
:1004100008956624552444243324222411240024DE
:1004200040E452E46FE06AD012F06394FCCF6AD0EB
:1004300040EA56E861E062D012F05394FCCF62D0FB
:1004400040E157E260E05AD012F04394FCCF5AD01A
:1004500048EE53E053D012F03394FCCF53D044E62F
:1004600050E04CD012F02394FCCF4CD04AE046D060
:1004700012F01394FCCF46D041E040D012F0039428
:10048000FCCFDD24EE24FF24089511270027DA167F
:10049000EB06F10640F4DF92EF92AF93BF93EF903B
:1004A000DF90BF91AF917D2C8E2C9F2C1197A117BF
:1004B000B10729F0D70CE81CF91C011FF7CF0895EC
:1004C00011272227AA27BB27D718E808F908010B0C
:1004D00018F01196211FF8CFDA2EEB2EF22E089588
:1004E0000695F794E794D7940895FADFF9DF089515
:1004F000F7DFFBDF0895F9DFFBDF0895D41AE50A83
:10050000F60A0895D40EE51EF61E089526E02A95F3
:10051000F1F708952BEE2A95F1F70895AFE0B7E2D1
:1005200022271197A217B207E1F70895AFEFBFEFA7
:1005300022271197A217B207E1F708951FE0F6DF0F
:100540001A951030E1F70895C29818B31370186027
:1005500007D00895C29A18B313701C6001D0089593
:10056000D5DFC39A3F93307F312B38BBCFDFC398A1
:10057000CDDFC39A3F913295307F312B38BBC6DF38
:10058000C398C8DFC7DF08955D9BFECF08952EBBDB
:100590001DBBE199FECFE29AE19AC0DFBFDF08956B
:1005A0002EBBE199FECFE09A2DB3089511E02227EA
:1005B0008030D1F0813091F0823051F0833021F0E1
:1005C000569547955695479556954795569547950F
:1005D00056954795569547955695479556954795FF
:1005E00056954795569547954117520710F444275D
:1005F00055270895869908C091DF869905C040D097
:1006000004D01F911F914ECD0895869BFECF86DFAB
:10061000869BFBCF0895B8DF10E1612A6CB8B4DF88
:1006200010E2512A5CB8B0DF10E3412A4CB8ACDFCD
:1006300010E4312A3CB8A8DF10E5212A2CB8A4DF49
:1006400010E6112A1CB8A0DF10E7012A0CB89CDFC5
:1006500008953EE47FDF3AE37DDF30E3350D7ADF56
:1006600030E3340D77DF30E3330D74DF30E3320DE8
:1006700071DF30E3310D6EDF30E3300D6BDF089555
:10068000D72CE82CF92CC5DE30E85EDFE2DFDA2C6F
:10069000EB2CFC2CBEDE30EC57DFDBDF0895F8944A
:1006A00013E0F11611F0F3941895909A949A959A94
:1006B00010E01EBD1F911F914BCD7CB48DB49F2CBB
:1006C00010E81BBF1895DCB4EDB4F894909A949A96
:1006D000959A10E01EBD1F911F91AD2CBE2CCF2C02
:1006E000D718E808F908903011F01FEF01C01EE19B
:1006F0002227D116E206F20610F07CDF38CD8030DA
:1007000009F031C0903011F099272DC086992BC087
:1007100005DF869928C02DE143DF243641F41FEF21
:100720002DE135DFE8EDF7E068DE6FDFBBCC172D9C
:1007300028E02DDF182D29E02ADF1A2D2BE027DFF6
:100740001B2D2EE024DF1D2D22E121DF1E2D27E1B0
:100750001EDF14E62DE11BDF93DF57DFE8ECF7E047
:100760004CDEECDE9FCCE8E9F7E047DEC3950CDF1A
:1007700011ED1CB909DFE8CC432026204553522057
:10078000B365702E20312E30A87065E365BB3A202A
:10079000B6E3B8BF652E2E2E4378203C206D696EDF
:1007A0004553523E206D61783C302C3031204FBC97
:1007B0003E32302C30204FBC4378203E206D617893
:1007C000B8BBB8204BA42020A86FBE7061B3BA613B
:1007D000B3BABBC6C065BD61A86FBE7061B3BA6174
:1007E00063B2706FC165BD61A461BC65BDB8BF6512
:1007F000B261BF617065C621B6E3B8BF652E2E2E0B
:00000001FF
